:020000040000FA
:020000000C28CA
:08000800A0000308A10021087B
:100010008300A00E200E090083128501073099008D
:1000200083169F0195010F308500FF2390008F30CC
:1000300081008312851605160A30A500640064301D
:10004000C82005126430C8200516A50B1E28BE2046
:100050006400A710352003192E28B5206400A714CA
:10006000352003192828B520282827102711A7187C
:100070003C28051827153F28000085182715271D3F
:1000800068286B20031968282508031D68286B2041
:100090000319682825080A3A031D682805122A3022
:1000A00084008001A718800A840A6B20031968283D
:1000B00025088000840A0408333A031D55282714B4
:1000C0006B20031968282508800005160311080015
:1000D000051603150800A501822003197E28A50D29
:1000E000822003197E28A50D822003197E28A50DE4
:1000F000822003197E28A50D0311080027187B28EC
:1001000003150800A601A3012711A7188A280518BE
:1001100027158D28000085182715271D9228A30F65
:100120008428B1282308143C0318B12823084B3C29
:100130000318A60AA2012711A718A1280518271538
:10014000A4280000851827152719A928A20F9B2885
:10015000B12822084B3C0318B1282608FF3E0311A2
:10016000B4282608FF3E031508002A308400000842
:10017000D120840A0408343A031DB7280D30D92051
:100180000A30D928A030A3000000A30BC42808001F
:10019000A200FA30A3000000A30BCB28A20BC928B1
:1001A0000800A4000F302405F63E0318073E3A3E2F
:1001B000D928A8000830A900E820A80C0318E228D4
:1001C000E820E428EA200000A90BDD28EA20080046
:1001D0008512EC288516EC281630A3000000A30B2E
:0401E000EE280800FD
:02400E00CC3FA5
:00000001FF
